:020000020000FC
:020000000DC031
:04000A00639518954D
:10001A00E6C00FEF07BB0FEF08BB0FE501BB00E01F
:10002A0002BB0FED0DBF00E808B900E205BF02E010
:10003A0000BF04E003BF0CE706BF00E00FBD07E006
:10004A000EBD01E809BF002741E051E0662771E0D3
:10005A009924AA24BB24CC24DD24EE24FF247894FA
:10006A008895FECF00E002BB713051F0723069F022
:10007A00733081F07430B1F07530E1F07630F9F018
:10008A00092D22D008BB909A08950A2D1DD008BBCD
:10009A00919A08950B2D18D0813009F4005808BBA5
:1000AA00929A08950C2D10D0803009F4005808BB9C
:1000BA00939A08950D2D08D008BB949A08950E2D91
:1000CA0003D008BB969A08950030A1F00130A1F040
:1000DA000230A1F00330A1F00430A1F00530A1F004
:1000EA000630A1F00730A1F00830A1F00930A1F0E4
:1000FA0007EF089500EC089509EF089504EA0895BA
:10010A0000EB089509E9089502E9089502E80895BF
:10011A0008EF089500E8089500E90895362F1CB500
:10012A002DB566276DBD6CBD88279924AA24BB24EA
:10013A00CC24DD24EE24FF24103806E9200708E940
:10014A00300750F00FEFF02EE02ED02EC02EB02E3A
:10015A00A02E902E8FEF42C0103402E420070FE049
:10016A00300728F0105422443F40F394F5CF103A58
:10017A0006E8200701E0300728F0105A26483140E7
:10018A00E394F5CF103107E2200700E0300728F0AA
:10019A00105127423040D394F5CF183E03E0200790
:1001AA0020F0185E2340C394F8CF143600E02007ED
:1001BA0020F014562040B394F8CF1A3018F01A5091
:1001CA00A394FBCF912E0027F01641F09A2CAB2C6A
:1001DA00BC2CCD2CDE2CEF2CFF248395089542DF16
:1001EA007A9509F476E04A9529F44DE75A9511F47F
:0601FA0055E094DF1895AA
:00000001FF
